BL51 BANKED LINKER/LOCATER V5.03                                                        04/25/2016  22:03:29  PAGE 1


BL51 BANKED LINKER/LOCATER V5.03, INVOKED BY:
C:\KEIL\C51\BIN\BL51.EXE main.obj, i2c.obj TO 99秒计数器 RAMSIZE (256)


MEMORY MODEL: SMALL


INPUT MODULES INCLUDED:
  main.obj (MAIN)
  i2c.obj (I2C)
  C:\KEIL\C51\LIB\C51S.LIB (?C_STARTUP)
  C:\KEIL\C51\LIB\C51S.LIB (?C?UIDIV)


LINK MAP OF MODULE:  99秒计数器 (MAIN)


            TYPE    BASE      LENGTH    RELOCATION   SEGMENT NAME
            -----------------------------------------------------

            * * * * * * *   D A T A   M E M O R Y   * * * * * * *
            REG     0000H     0008H     ABSOLUTE     "REG BANK 0"
            DATA    0008H     0006H     UNIT         ?DT?MAIN
            DATA    000EH     0001H     UNIT         _DATA_GROUP_
            IDATA   000FH     0001H     UNIT         ?STACK

            * * * * * * *   C O D E   M E M O R Y   * * * * * * *
            CODE    0000H     0003H     ABSOLUTE     
            CODE    0003H     0001H     UNIT         ?PR?DELAY?I2C
                    0004H     0007H                  *** GAP ***
            CODE    000BH     0003H     ABSOLUTE     
            CODE    000EH     0055H     UNIT         ?C?LIB_CODE
            CODE    0063H     0052H     UNIT         ?PR?_DISPLAY?MAIN
            CODE    00B5H     0035H     UNIT         ?PR?TIME0?MAIN
            CODE    00EAH     002CH     UNIT         ?PR?MAIN?MAIN
            CODE    0116H     0023H     UNIT         ?PR?_WRITE_BYTE?I2C
            CODE    0139H     0022H     UNIT         ?PR?_READ_AT24C02?I2C
            CODE    015BH     0020H     UNIT         ?PR?ACK?I2C
            CODE    017BH     0020H     UNIT         ?PR?READ_BYTE?I2C
            CODE    019BH     0018H     UNIT         ?PR?_WRITE_AT24C02?I2C
            CODE    01B3H     0010H     UNIT         ?PR?INIT_TIME0?MAIN
            CODE    01C3H     0010H     UNIT         ?CO?MAIN
            CODE    01D3H     000EH     UNIT         ?PR?_DELAY1?MAIN
            CODE    01E1H     000CH     UNIT         ?PR?START?I2C
            CODE    01EDH     000CH     UNIT         ?PR?STOP?I2C
            CODE    01F9H     000CH     UNIT         ?PR?NACK?I2C
            CODE    0205H     000CH     UNIT         ?C_C51STARTUP



OVERLAY MAP OF MODULE:   99秒计数器 (MAIN)


SEGMENT                          DATA_GROUP 
  +--> CALLED SEGMENT          START    LENGTH
----------------------------------------------
?C_C51STARTUP                  -----    -----
  +--> ?PR?MAIN?MAIN
BL51 BANKED LINKER/LOCATER V5.03                                                      04/25/2016  22:03:29  PAGE 2



?PR?MAIN?MAIN                  -----    -----
  +--> ?PR?START?I2C
  +--> ?PR?_READ_AT24C02?I2C
  +--> ?PR?INIT_TIME0?MAIN
  +--> ?PR?_DISPLAY?MAIN
  +--> ?PR?_WRITE_AT24C02?I2C

?PR?START?I2C                  -----    -----
  +--> ?PR?DELAY?I2C

?PR?_READ_AT24C02?I2C          -----    -----
  +--> ?PR?ACK?I2C
  +--> ?PR?_WRITE_BYTE?I2C
  +--> ?PR?START?I2C
  +--> ?PR?READ_BYTE?I2C
  +--> ?PR?NACK?I2C
  +--> ?PR?STOP?I2C

?PR?ACK?I2C                    000EH    0001H
  +--> ?PR?START?I2C
  +--> ?PR?_WRITE_BYTE?I2C
  +--> ?PR?DELAY?I2C

?PR?_WRITE_BYTE?I2C            -----    -----
  +--> ?PR?DELAY?I2C

?PR?READ_BYTE?I2C              -----    -----
  +--> ?PR?DELAY?I2C

?PR?NACK?I2C                   -----    -----
  +--> ?PR?DELAY?I2C

?PR?STOP?I2C                   -----    -----
  +--> ?PR?DELAY?I2C

?PR?_DISPLAY?MAIN              -----    -----
  +--> ?CO?MAIN
  +--> ?PR?_DELAY1?MAIN

?PR?_WRITE_AT24C02?I2C         -----    -----
  +--> ?PR?ACK?I2C
  +--> ?PR?_WRITE_BYTE?I2C
  +--> ?PR?STOP?I2C



SYMBOL TABLE OF MODULE:  99秒计数器 (MAIN)

  VALUE           TYPE          NAME
  ----------------------------------

  -------         MODULE        MAIN
  C:0000H         SYMBOL        _ICE_DUMMY_
  D:0080H         PUBLIC        P0
  D:0090H         PUBLIC        P1
  D:00A0H         PUBLIC        P2
BL51 BANKED LINKER/LOCATER V5.03                                                      04/25/2016  22:03:29  PAGE 3


  D:00B0H         PUBLIC        P3
  B:00A8H.7       PUBLIC        EA
  D:00A8H         PUBLIC        IE
  D:0008H         PUBLIC        disnum
  D:00B8H         PUBLIC        IP
  C:01D3H         PUBLIC        _delay1
  C:00EAH         PUBLIC        main
  B:00A0H.6       PUBLIC        dula
  B:00A0H.7       PUBLIC        wela
  D:0098H         PUBLIC        SCON
  D:0089H         PUBLIC        TMOD
  D:0088H         PUBLIC        TCON
  C:01C3H         PUBLIC        table_du
  B:00A8H.1       PUBLIC        ET0
  D:008CH         PUBLIC        TH0
  D:008AH         PUBLIC        TL0
  D:000AH         PUBLIC        num
  B:0088H.4       PUBLIC        TR0
  C:0063H         PUBLIC        _display
  C:00B5H         PUBLIC        time0
  D:00C8H         PUBLIC        T2CON
  D:000CH         PUBLIC        t
  C:01B3H         PUBLIC        init_time0
  D:00D0H         PUBLIC        PSW
  -------         PROC          _DELAY1
  D:0007H         SYMBOL        x
  -------         DO            
  D:0007H         SYMBOL        a
  D:0006H         SYMBOL        b
  -------         ENDDO         
  C:01D3H         LINE#         18
  C:01D3H         LINE#         19
  C:01D3H         LINE#         21
  C:01D9H         LINE#         22
  C:01E0H         LINE#         23
  -------         ENDPROC       _DELAY1
  -------         PROC          _DISPLAY
  D:0002H         SYMBOL        disnum
  C:0063H         LINE#         25
  C:0067H         LINE#         26
  C:0067H         LINE#         27
  C:007CH         LINE#         28
  C:007EH         LINE#         29
  C:0080H         LINE#         30
  C:0083H         LINE#         31
  C:0085H         LINE#         32
  C:0087H         LINE#         33
  C:008CH         LINE#         35
  C:00A5H         LINE#         36
  C:00A7H         LINE#         37
  C:00A9H         LINE#         38
  C:00ACH         LINE#         39
  C:00AEH         LINE#         40
  C:00B0H         LINE#         41
  -------         ENDPROC       _DISPLAY
  -------         PROC          INIT_TIME0
  C:01B3H         LINE#         44
BL51 BANKED LINKER/LOCATER V5.03                                                      04/25/2016  22:03:29  PAGE 4


  C:01B3H         LINE#         45
  C:01B3H         LINE#         46
  C:01B5H         LINE#         47
  C:01B7H         LINE#         48
  C:01BAH         LINE#         49
  C:01BDH         LINE#         50
  C:01C0H         LINE#         51
  C:01C2H         LINE#         52
  -------         ENDPROC       INIT_TIME0
  -------         PROC          MAIN
  C:00EAH         LINE#         54
  C:00EAH         LINE#         55
  C:00EAH         LINE#         56
  C:00EDH         LINE#         57
  C:00F7H         LINE#         58
  C:00FAH         LINE#         59
  C:00FAH         LINE#         60
  C:00FAH         LINE#         61
  C:0101H         LINE#         62
  C:0109H         LINE#         63
  C:0109H         LINE#         64
  C:010DH         LINE#         65
  C:0114H         LINE#         66
  C:0114H         LINE#         67
  -------         ENDPROC       MAIN
  -------         PROC          TIME0
  C:00B5H         LINE#         70
  C:00B7H         LINE#         72
  C:00BAH         LINE#         73
  C:00BDH         LINE#         74
  C:00C5H         LINE#         75
  C:00CBH         LINE#         76
  C:00CBH         LINE#         77
  C:00CFH         LINE#         78
  C:00D7H         LINE#         79
  C:00DDH         LINE#         80
  C:00E3H         LINE#         81
  C:00E7H         LINE#         82
  C:00E7H         LINE#         83
  -------         ENDPROC       TIME0
  -------         ENDMOD        MAIN

  -------         MODULE        I2C
  C:0000H         SYMBOL        _ICE_DUMMY_
  D:0090H         PUBLIC        P1
  D:00A0H         PUBLIC        P2
  D:00B0H         PUBLIC        P3
  D:00A8H         PUBLIC        IE
  C:0003H         PUBLIC        delay
  D:00B8H         PUBLIC        IP
  B:00D0H.7       PUBLIC        CY
  C:01F9H         PUBLIC        nack
  C:0116H         PUBLIC        _write_byte
  C:0163H         PUBLIC        ack
  C:01E1H         PUBLIC        start
  D:0098H         PUBLIC        SCON
  C:017BH         PUBLIC        read_byte
BL51 BANKED LINKER/LOCATER V5.03                                                      04/25/2016  22:03:29  PAGE 5


  D:0088H         PUBLIC        TCON
  C:01EDH         PUBLIC        stop
  B:00A0H.0       PUBLIC        SDA
  C:0139H         PUBLIC        _read_at24c02
  B:00A0H.1       PUBLIC        SCL
  D:00C8H         PUBLIC        T2CON
  C:019BH         PUBLIC        _write_at24c02
  D:00D0H         PUBLIC        PSW
  -------         PROC          DELAY
  C:0003H         LINE#         2
  C:0003H         LINE#         3
  C:0003H         LINE#         5
  -------         ENDPROC       DELAY
  -------         PROC          START
  C:01E1H         LINE#         6
  C:01E1H         LINE#         7
  C:01E1H         LINE#         8
  C:01E3H         LINE#         9
  C:01E5H         LINE#         10
  C:01E8H         LINE#         11
  C:01EAH         LINE#         12
  -------         ENDPROC       START
  -------         PROC          STOP
  C:01EDH         LINE#         15
  C:01EDH         LINE#         16
  C:01EDH         LINE#         17
  C:01EFH         LINE#         18
  C:01F1H         LINE#         19
  C:01F4H         LINE#         20
  C:01F6H         LINE#         21
  -------         ENDPROC       STOP
  -------         PROC          L?0018
  -------         ENDPROC       L?0018
  -------         PROC          ACK
  -------         DO            
  D:000EH         SYMBOL        i
  -------         ENDDO         
  C:0163H         LINE#         24
  C:0163H         LINE#         25
  C:0163H         LINE#         27
  C:0165H         LINE#         28
  C:0168H         LINE#         29
  C:0176H         LINE#         30
  C:0178H         LINE#         31
  -------         ENDPROC       ACK
  -------         PROC          NACK
  C:01F9H         LINE#         34
  C:01F9H         LINE#         35
  C:01F9H         LINE#         36
  C:01FBH         LINE#         37
  C:01FEH         LINE#         38
  C:0200H         LINE#         39
  C:0202H         LINE#         40
  -------         ENDPROC       NACK
  -------         PROC          _WRITE_BYTE
  D:0007H         SYMBOL        date
  -------         DO            
BL51 BANKED LINKER/LOCATER V5.03                                                      04/25/2016  22:03:29  PAGE 6


  D:0006H         SYMBOL        i
  D:0007H         SYMBOL        temp
  -------         ENDDO         
  C:0116H         LINE#         43
  C:0116H         LINE#         44
  C:0116H         LINE#         46
  C:0116H         LINE#         47
  C:0118H         LINE#         48
  C:0118H         LINE#         49
  C:011CH         LINE#         50
  C:011EH         LINE#         51
  C:0121H         LINE#         52
  C:0123H         LINE#         53
  C:0126H         LINE#         54
  C:0128H         LINE#         55
  C:012BH         LINE#         56
  C:012FH         LINE#         57
  C:0131H         LINE#         58
  C:0134H         LINE#         59
  C:0136H         LINE#         60
  -------         ENDPROC       _WRITE_BYTE
  -------         PROC          READ_BYTE
  -------         DO            
  D:0006H         SYMBOL        i
  D:0005H         SYMBOL        j
  D:0007H         SYMBOL        k
  -------         ENDDO         
  C:017BH         LINE#         63
  C:017BH         LINE#         64
  C:017BH         LINE#         66
  C:017DH         LINE#         67
  C:0180H         LINE#         68
  C:0182H         LINE#         69
  C:0182H         LINE#         70
  C:0184H         LINE#         71
  C:0187H         LINE#         72
  C:018CH         LINE#         73
  C:0191H         LINE#         74
  C:0193H         LINE#         75
  C:0196H         LINE#         76
  C:019AH         LINE#         77
  C:019AH         LINE#         78
  -------         ENDPROC       READ_BYTE
  -------         PROC          _WRITE_AT24C02
  D:0004H         SYMBOL        address
  D:0005H         SYMBOL        date
  C:019BH         LINE#         80
  C:019DH         LINE#         81
  C:019DH         LINE#         82
  C:019DH         LINE#         83
  C:019DH         LINE#         84
  C:01A0H         LINE#         85
  C:01A5H         LINE#         86
  C:01A8H         LINE#         87
  C:01ADH         LINE#         88
  C:01B0H         LINE#         89
  -------         ENDPROC       _WRITE_AT24C02
BL51 BANKED LINKER/LOCATER V5.03                                                      04/25/2016  22:03:29  PAGE 7


  -------         PROC          _READ_AT24C02
  D:0005H         SYMBOL        address
  -------         DO            
  D:0007H         SYMBOL        date
  -------         ENDDO         
  C:0139H         LINE#         92
  C:013BH         LINE#         93
  C:013BH         LINE#         95
  C:013BH         LINE#         96
  C:013BH         LINE#         97
  C:013EH         LINE#         98
  C:0143H         LINE#         99
  C:0146H         LINE#         100
  C:0149H         LINE#         101
  C:014EH         LINE#         102
  C:0151H         LINE#         103
  C:0154H         LINE#         104
  C:0157H         LINE#         105
  C:015AH         LINE#         106
  C:015AH         LINE#         107
  -------         ENDPROC       _READ_AT24C02
  -------         ENDMOD        I2C

  -------         MODULE        ?C?UIDIV
  C:000EH         PUBLIC        ?C?UIDIV
  -------         ENDMOD        ?C?UIDIV

Program Size: data=16.0 xdata=0 code=522
LINK/LOCATE RUN COMPLETE.  0 WARNING(S),  0 ERROR(S)
